:020000040000FA
:060000008316031315280E
:08000800BA000308BC00040863
:10001000BB000A08BD0053213D088A003B0884004C
:100020003C088300BA0E3A0E090002309F002F30C0
:100030008500D7308100C0308600073087008312EA
:10004000031380309F00EF308500FF308600F730CB
:100050008700203084008001840A3E300402031DA2
:100060002B280230A222AA000330A222AB004B228E
:10007000F030A400B0308100A0308B000608C039F9
:100080000319D728861FF528061F2929702820184C
:100090006428A0187B28201D5528B908031D8A282C
:1000A000F430B900A60B8A2820112F082C0203185F
:1000B0008A280030A222A5002014A0102011871544
:1000C0000512F430B9008E282014A01020118715D5
:1000D0000512B908031D8E28F430B900A50B8E282F
:1000E0000130A222A6002010A014201187110516AD
:1000F000F430B9008E282010A014201187110516A5
:10010000B908031D8E28F430B900A60B8E282015DF
:100110000A30A600A01020108711051234083302FF
:100120000318A228071CB028FF3A013EA200CF30D6
:100130002404FF3AFC30031DFE3022050319B028C9
:100140004522B228871CB028A200CF302404FF3AF1
:10015000FC30031DFE3022050319B0283F22B228CF
:100160003030A404320831020318C628211CD428D8
:10017000FF3A013EA2003F302404FF3AFC30031D49
:10018000FE3022050319D42839224728A11CD4287F
:10019000A2003F302404FF3AFC30031DFE3022054C
:1001A0000319D42833224728C030A4044728201636
:1001B0001930A5002530840000308B13AF220D309C
:1001C000A600263084000130AF228B17F430B9002E
:1001D0001930A200B908031DE828F430B900253011
:1001E000A200B908031DEF28E6282016861FF5286F
:1001F000061B0F293230A2008715F4309D22061B02
:100200000329A20BFC283230A5002208A5020319FD
:10021000A50A2530840000308B13AF228B1787117D
:10022000861B27293230A2000516F4309D22861B3A
:100230001B29A20B14293230A6002208A60203199A
:10024000A60A2630840001308B13AF228B170512CB
:10025000F828A016061F2929861B3D29071C3229CC
:1002600045222C29F030A404861B3D29871C3A29FD
:100270003F223429F030A4042C29F030A404061BBA
:100280005029A11C452933223F29F030A404061B24
:100290005029211C4D2939224729F030A4043F2937
:1002A000F030A4042C290B1D0800B03081000B1184
:1002B00076225622B808031DB803B908031DB903F6
:1002C0000F22201AFE2924083F38FF3A031D6D290A
:1002D00087170000000007178629B508031D7E292F
:1002E000A41B772907170000000087138229241B0D
:1002F0007E29871700000000071382298717000056
:1003000000000717B50A013035020318B5012408AB
:10031000CF38FF3A031D9129871600000000071609
:10032000AA29B608031DA229A41A9B2907160000B2
:1003300000008712A629241AA229871600000000AF
:100340000712A6298716000000000716B60A01301A
:1003500036020318B601A01A0800A7080319CD2910
:10036000A703201BB729061BD3292017BD29061B6D
:10037000C9292017A708031DD429AA0A0A302A026E
:100380000318AA012A3084000230AF226130A7008E
:10039000D4292013F430A700D429061BD329201711
:1003A000F430A700D4292013A8080319F529A803BD
:1003B000A01BDE29861BFB29A017E429861BF12937
:1003C000A017A808031DFC29AB0A0A302B02033032
:1003D0000318AB002B3084000330AF226130A8003B
:1003E000FC29A013F430A800FC29861BFB29A017C8
:1003F000F430A800FC29A0134B220800A70B08002A
:100400003230AA002208AA02AB010A302A02031CD9
:100410000C2AAA00AB0A052A3130A7000800A90A55
:100420003030A300FF308600A708031D1C2AA8084F
:10043000031D1C2A2D301D2A2A3084002918222A47
:100440002312242A840AA31200080F3923048600E9
:100450009322A114211407190800291C312AA11084
:10046000080021100800241B372A24179C22A413FB
:100470000800A41B3D2AA4179C2224130800241A58
:10048000432A24169C22A4120800A41A492AA4165E
:100490009C222412080003102B08AC00AC0D2C0881
:1004A000AC0DAC0DAC072A08AC070800AF01AE01DB
:1004B0003008E63CAD000318692AFF3A013EAD0062
:1004C000093C031C662A6430AD076F2A6D30AD000D
:1004D0006F2AAF00633C03186F2A6330AD000A3007
:1004E0002D02031C0800AD00AE0A6F2A81308C2259
:1004F000B400932289308C22B300932291308C2255
:10050000B200932299308C22B1009322A1308C2228
:10051000B00080309F0008009F0093221F151F1914
:100520008F2A1E0808001730B7000000B70B952A65
:1005300000000000000008001930B800B808031DD2
:100540009E2A0800831203178D00831603178C134D
:100550000C14831203170C08831203130800831270
:1005600003178D000008831203178C0083160317EE
:100570008C130C1555308D00AA308D008C140000A2
:0C0580008C18BF2A0C1183120313080012
:02400E00323F3F
:0842000019000D000500080083
:00000001FF
